:100000009F2864001120031801281C2008308F004D
:100010001D2011208E0C0C288F0B08281D200E0887
:100020000800220884002008841780048413000537
:100030001F192006FF3E08001F171F0D06398C00F0
:100040002B208D008C0A2B201F1F7E281F138C0055
:10005000023095207E2800308A000C088207013487
:1000600075340334153400343C340C34D9348F00E7
:100070002208840020095E2084138F0803199A281F
:10008000F03091000E0880389000F0309103031991
:10009000910003198F0303199A284E286120030148
:1000A0000C1820088E1F20088E0803190301900FDA
:1000B0005B28800642285C280000452884178005BC
:1000C0009A280D080C0403198C0A80300C1A8D062E
:1000D0000C198D068C188D060D0D8C0D8D0D9A2822
:1000E0008F018E00FF308E07031C8F07031C9A2898
:1000F00003308D00DF307E2072288D01E83E8C00B9
:100100008D09FC30031C87288C07031884288C0772
:1001100064008D0F84280C188D288C1C91280000F9
:100120009128080003108D0C8C0CFF3E03189228B8
:100130000C089A28831303138312640008008316A3
:10014000850101308600831206128316061283127F
:1001500006138316061383128612831686128312E1
:1001600086108316861083120611831606118312D9
:1001700086118316861105308312A2000830A00074
:1001800073308E000A30372032308E000A3037202C
:100190000630A2000130A00004309F0001205A3C2C
:1001A000031DCE280120A40064002408413C031D47
:1001B000DA281B2164002408423C031DE0287D212D
:1001C00064002408433C031DE6284C2164002408F5
:1001D000443C031DEC28AE2164002408453C031D6B
:1001E000FD280530A2000830A00073308E000A30D0
:1001F000372032308E000A30372064002408463C15
:10020000031D1A290612831606128312061383167B
:1002100006138312861283168612831286108316A3
:100220008610831206118316061183128611831617
:1002300086118312C8280616831606128312061723
:1002400083160613831201308F002C307120640056
:1002500005182B2927290612831606128312061366
:1002600083160613831286148316861083120615CE
:1002700083160611831201308F002C307120640028
:10028000851843293F29861083168610831206118C
:1002900083160611831208000616831606128312AF
:1002A000861683168612831201308F002C3071203F
:1002B000640005185C295829061283160612831259
:1002C0008612831686128312861483168610831272
:1002D000061583160611831201308F002C30712011
:1002E000640085187429702986108316861083127D
:1002F00006118316061183120800061683160612CD
:100300008312861683168612831201308F002C30DA
:100310007120640005188D2989290612831606129A
:100320008312861283168612831286148316861011
:100330008312861583168611831201308F002C30AC
:10034000712064008518A529A129861083168610BE
:1003500083128611831686118312080006168316EF
:1003600006128312061783160613831201308F00BC
:100370002C30712064000518BE29BA290612831694
:10038000061283120613831606138312861483162D
:1003900086108312861583168611831201308F0012
:1003A0002C30712064008518D629D2298610831636
:1003B000861083128611831686118312080063004B
:0203C000DF2933
:02400E00F53F7C
:00000001FF
